:100000000C94D2030C9419040C9419040C94190444
:100010000C9419040C9419040C9419040C941904EC
:100020000C9419040C9419040C94B50E0C94870FBD
:100030000C9419040C9419040C9419040C941904CC
:100040000C9419040C9443230C9419040C94190473
:100050000C9419040C94D71C0C9419040C941904D6
:100060000C9419040C9419040C9419040C9419049C
:100070000C9419040C9419040C9419040C9419048C
:100080000C9419040C9419040C9419040C9419047C
:100090000C9419040C9419040C9419040C9419046C
:1000A0000C9419040C9419040C941904F40F1610F0
:1000B0000411161004115B107E100411D310E61009
:1000C000B513B513E413E4131A143A146B156B1536
:1000D00045146B15F514F5145C156B156B1565154A
:1000E0000215021502150215021502150215021558
:1000F0000215021502150215021502150215021548
:100100001415211528152F15391502E002E20001FA
:10011000E201E00002620001620262016200350059
:100120002E0030006400015400001E001400040082
:100130001D00000004521F001A0016001B00E300FF
:10014000E1002000080007000600E0002C0021006C
:10015000150009001900E2000552220017000A00EC
:100160000500000029004C002A0000002B000000C0
:100170000652470039000000530000000000230031
:100180001C000B00110000004900240018000D00A5
:100190001000E600013025000C000E003600E400DF
:1001A0002800260012000F003700E700E5002700B6
:1001B000130033003800460004522D002F00340095
:1001C000310048000000210222021A00080001004C
:1001D000000034020500040004000000045236024E
:1001E000080018001C00E3000252370213000C0044
:1001F0001B00E0002C002602120008003700E2007D
:1002000005522702080036000E00000029004C00AD
:100210002A0000002B0000000652470039000000B1
:100220005300000000001F022302060034000000FB
:1002300049002E02190017001400035201002D007E
:10024000070016000A00E400280038000F0015001F
:100250000B00E700025225020D00110009004600C4
:1002600004522E001D00100006004800000020026D
:1002700035001A020802010000001E0005020402F7
:100280000402010001001F00080218021C02E30220
:100290000100200013020C021B02E00201002100F9
:1002A000120208023302E2020100220008023300B7
:1002B0000E02000001000100010000002B020000FE
:1002C0000100010001000000010000000100230006
:1002D0001E02060238020000010024001902170263
:1002E0001402E60201002500070216020A02E402D7
:1002F000010026000F0215020B02E7020100270091
:100300000D02110209020100010001001D0210028C
:10031000060201000000210222021A00080001006A
:1003200000003402310204003100000004523602A1
:10033000080018002F02E3000252370224020C00CA
:100340003002E0002D022F00120022143700E200DC
:1003500005523000080036003502000029004C002C
:100360002A0000002B000000065247003900000060
:100370005300000000001F022302060034000000AA
:1003800049002E02190017001400010001002D0081
:10039000070016000A00E400280038000F001500CE
:1003A0000B00E700025225020D0011000900460073
:1003B00004522E001D00100006004800000000003E
:1003C000000000000000000000003A0000000000F3
:1003D0007A00000001003B00000000007B000100EB
:1003E00001003C00000000007C00010000003D0016
:1003F000000000007D00010000003E000000000041
:10040000000000000000A800A9000000AA000000F1
:1004100000000000000000000000000000003F009D
:100420004B004E0000000000000040004A00500059
:1004300000000100010041005200510000000100D5
:10044000000042004D004F00000001000100430089
:100450004400450000000000010000000000000012
:10046000000000000000000000000000000000008C
:10047000000000000000000000000000000000007C
:10048000000000000000010001000000000000006A
:10049000000001000000000000000000000001005A
:1004A000010000000000000000000000000000004B
:1004B000000000000000000000000000000000003C
:1004C000000000000000000000000000000000002C
:1004D000000057005F005C005900620000005600F9
:1004E00060005D005A0000305800540061005E005A
:1004F0005B008500010055000000000000000000C6
:1005000000000000000000000000000000000000EB
:1005100000000000000000000000000000000000DB
:1005200000000000000000000000000000000100CA
:1005300001000000000000000000010000000000B9
:1005400000000000000001000000000000000000AA
:10055000000000000000000000000000000000009B
:10056000010000000000000000000000000000008A
:10057000000000000000000000000000F400F20095
:100580000000010000000000F000F1000000010088
:1005900000000000F500F300000001000100000071
:1005A000F900FA0000000000000000000000000058
:1005B00000000000000016034500720067006F0095
:1005C00044006F007800200045005A000000160328
:1005D0004500720067006F0044006F007800200043
:1005E00045005A0000000403090409026D000401DB
:1005F00000A0FA0904000001030101000921110112
:100600000001223F000705810308000A09040100D8
:100610000103010200092111010001224D0007051B
:10062000820308000A0904020001030000000921F6
:10063000110100012236000705830308000A09049E
:10064000030001030000000921110100012239000B
:10065000070584031000011201100100000008EDDD
:10066000FE071301000102000105010906A10105B1
:100670000719E029E7150025019508750181020594
:1006800008190129059505750191029501750391D8
:100690000105071900297715002501957875018155
:1006A00002C005010980A101850216010026B700DC
:1006B0001A01002AB700751095018100C0050C09C8
:1006C00001A1018503160100269C021A01002A9C43
:1006D00002751095018100C005010902A1010901FF
:1006E000A1000509190129051500250195057501C8
:1006F00081029501750381010501093009311581D8
:10070000257F95027508810609381581257F950199
:1007100075088106050C0A38021581257F9501753B
:10072000088106C0C005010906A101050719E029D5
:10073000E71500250195087501810295017508816D
:1007400001050819012905950575019102950175A5
:100750000391010507190029FF150025FF9506756E
:10076000088100C00000000000000000000000013F
:100770000204060A0F17202C3A4A5D71879DB3C701
:10078000DAE9F5FCFFFCF5E9DAC7B39D87715D4A4C
:100790003A2C20170F0A0604020100000000000096
:1007A0000000000011241FBECFEFDAE0DEBFCDBF96
:1007B00004B603FE27C08091FB019091FC01A0913B
:1007C000FD01B091FE018730904BA740B04BD1F4B2
:1007D0001092FB011092FC011092FD011092FE019B
:1007E00014BE84B7877F84BF0FB6F894A895809114
:1007F0006000886180936000109260000FBEE0E0AE
:10080000FFE3099511E0A0E0B1E0E2E3FAE402C001
:1008100005900D92A433B107D9F721E0A4E3B1E02C
:1008200001C01D92AB3FB207E1F70E94F60B0C949A
:1008300017250C940000662319F0613041F017C0B1
:10084000FC018281811116C084E191E00895FC01D0
:100850008281882331F084E00E94131A8FE091E0B6
:10086000089584E00E94341A8AE091E0089580E0BF
:1008700090E0089587E191E00895089508950C941B
:100880003E0456985E9825982D9826982E9827987D
:100890002F988FEF90E09093890080938800909339
:1008A0008B0080938A0090938D0080938C00259A12
:1008B0002D9A2FEF80E792E0215080409040E1F7A1
:1008C00000C00000269A2E9A2FEF80E792E0215078
:1008D00080409040E1F700C00000279A2F9A2FEF48
:1008E00080E792E0215080409040E1F700C0000096
:1008F00025982D982FEF80E792E02150804090407E
:10090000E1F700C0000026982E982FEF80E792E0D4
:10091000215080409040E1F700C0000027982F98B8
:1009200056985E9825982D9826982E9827982F9857
:10093000089589EA8093800089E08093810024985B
:100940002C983F988AB18F748AB96E98479A8BB168
:10095000806B8BB9769A0E9441040C943D0480E22E
:10096000809300018091340181110EC00E94FE0429
:1009700081E0809334012FEF83ED90E3215080409C
:100980009040E1F700C0000080E40E9404058093DD
:10099000000181112EC00E942E058093000181115B
:1009A00028C00E942E0580930001811122C08FE390
:1009B0000E942E058093000181111BC00E94260514
:1009C00080E40E94040580930001811112C08CE034
:1009D0000E942E058093000181110BC00E942E05FC
:1009E00080930001811105C08FE30E942E05809342
:1009F00000010E9426058091000108951092B9001F
:100A00008AE08093B800089594EA9093BC00909196
:100A1000BC0097FFFCCF9091B900987F983021F0EF
:100A2000903111F081E008958093BB0084E88093B9
:100A3000BC008091BC0087FFFCCF8091B900887F0B
:100A4000883111F0803471F780E0089584E9809353
:100A5000BC008091BC0084FDFCCF08958093BB0056
:100A600084E88093BC008091BC0087FFFCCF90910C
:100A7000B900987F81E0983209F480E0089584E815
:100A80008093BC008091BC0087FFFCCF8091BB00AD
:100A9000089580910001811115C080E40E94040531
:100AA0008093000181110CC082E10E942E05809389
:100AB0000001811105C08FEF0E942E058093000177
:100AC0000E94260584B1807F84B985B1807F85B975
:100AD0008AB1837F8AB98BB1837F8BB93E98469860
:100AE00008950E94AF04809300010E94490580B3DD
:100AF0008C7080BB81B3836F81BBA6E3B1E0E4E47B
:100B0000F1E08EE08E0F11921D928E13FCCF0C94AB
:100B10009904BF92CF92DF92EF92FF920F931F93AF
:100B2000CF93DF9380910001882379F08091350184
:100B30008F5F80933501811108C00E94AF048093BC
:100B40000001811102C00E94410406E311E0C0E0EF
:100B5000D0E0DD24D39482E0C82EEE24E394F12C7F
:100B6000C730D10500F580910001811164C080E497
:100B70000E94040580930001811112C082E10E944D
:100B80002E058093000181110BC0C7010C2E01C0FE
:100B9000880F0A94EAF780950E942E058093000141
:100BA0000E94260548C0CA30A1F028F4C83059F088
:100BB000C93061F005C0CC3089F070F0CD3089F0DB
:100BC000209A289810C0219A29980DC0229A2A9814
:100BD0000AC0239A2B9807C0529A01C0539A5B9877
:100BE00002C03E9A469890EA9A95F1F79FB179999A
:100BF00002C082E001C080E091709D25982B7C9915
:100C000002C084E001C080E0892B7D9902C038E0F9
:100C100001C030E0832B7E9902C020E101C020E0BA
:100C2000822B9FB19095991F9927991F9295990FA3
:100C3000907E892B0FC080910001811149C080E412
:100C40000E94040580930001882379F1B12C0E9451
:100C500026058B2DF8019081981719F08083C0929A
:100C600001010E94490521960F5F1F4FCE30D1052B
:100C700009F076CF80910101882361F18150809342
:100C80000101882339F08FE99FE00197F1F700C057
:100C9000000020C0A4E4B1E0E6E3F1E0CF01825F10
:100CA00091919D938E13FCCF15C083E10E942E0578
:100CB000809300018111CACF81E40E9404058093D2
:100CC00000018111C3CF0E943F05B82EB094BFCF61
:100CD00080E0C0CF0E943F0481E0DF91CF911F915F
:100CE0000F91FF90EF90DF90CF90BF900895E82F85
:100CF000F0E0EC5BFE4F8081089508950F931F9301
:100D0000CF93DF93C4E4D1E010E00C2F025F899110
:100D100090E00E944A1C180F0C13F9CF812FDF912D
:100D2000CF911F910F91089581E0089581E008957A
:100D30000C94960608950F931F93CF93DF938C0125
:100D4000FC01C081D181CE010E94CF1ABE010E9458
:100D50004407EC01B8010E949806882309F48DC06D
:100D6000F8018281882309F44AC080915D018111D4
:100D70001FC0C431F0E5DF0709F051C00E949A0698
:100D800081E080935D010E94A11C90935C0180939F
:100D90005B0110925401109256011092550110926D
:100DA00058011092570110925A011092590165C0D2
:100DB00080915B0190915C010E94AD1C883C910583
:100DC00070F480915401E82FF0E0EE0FFF1FEB5A12
:100DD000FE4FD183C0838F5F809354014EC0C438CF
:100DE00080E5D80721F0C538D04501F13AC0F801B7
:100DF0008281882341F01092520182E01EC0C438E3
:100E0000E0E5DE0759F580915201811106C086E2C6
:100E10000E94591286E20E94211382E01CC0C4384D
:100E2000F0E5DF0741F3C538D045D9F4F8018281F8
:100E3000882331F01092530180E20E9470131DC08C
:100E400080915301811106C087E20E94591287E206
:100E50000E94211380E20E9477130FC0C538D0454D
:100E600029F381E08093520180935301C801DF91FF
:100E7000CF911F910F910C94940680E0DF91CF9158
:100E80001F910F910895089596E0799FF001112424
:100E900094E5899FE00DF11D1124E60FF11DEE0F81
:100EA000FF1FE25EFE4F859194910895880F991F70
:100EB000FC01E256F040859194910895880F991FA6
:100EC000FC01E25EFE4F8591949108950F931F936C
:100ED000CF93DF93EC018115904350F5C11580E26B
:100EE000D80708F0C3C0CB3BD10590F4C83AD10570
:100EF00008F06AC0C53AD10508F05BC0C430D1051E
:100F000008F0D0C1219709F0CAC101E010E00AC27F
:100F1000CF3FD10511F008F0C5C1C03FD10508F0A1
:100F2000A2C0CE01805E9109089708F4BBC1B7C189
:100F3000C13090E5D90709F4A2C020F5C0318FE493
:100F4000D80770F4C11590E4D90708F094C0C11512
:100F500021E3D20708F0A3C1DD278E01106CE2C1A6
:100F6000C115D04509F09BC10E94D6158FEF94E3BF
:100F70002CE0815090402040E1F700C000000E942A
:100F8000FC1CD0C1C11597E5D90758F4C03121E543
:100F9000D20708F01CC1C43180E5D80708F475C039
:100FA0007EC1CE0190578115904108F078C1DF7065
:100FB00073C1C53AD10509F477C1C63AD10509F024
:100FC00076C102E810E4AEC1C83AD10509F472C195
:100FD000C93AD10509F471C1CA3AD10509F470C101
:100FE000CB3AD10509F46FC1CC3AD10509F46EC1F1
:100FF000CD3AD10509F46DC1C03BD10509F46CC1EE
:10100000CE3AD10509F46BC1CF3AD10509F46AC1D2
:10101000C13BD10509F469C1C23BD10509F468C1DE
:10102000C33BD10509F467C1C43BD10509F466C1CE
:10103000C53BD10509F465C1C63BD10509F464C1BE
:10104000C73BD10509F463C1C83BD10509F462C1AE
:10105000C93BD10509F461C1CA3BD10509F460C19E
:1010600000E014E45FC18E0110655CC1CE019F7089
:101070000E945E0758C1DF708E01106A53C18091D3
:10108000DA0181608093DA014DC10E94A11E8111B5
:1010900002C00E94871E0E94BE1E90E09093FB013A
:1010A0008093FA01C23080E5D80721F48091FA01DB
:1010B000816086C0C43090E5D90721F48091FA019F
:1010C00082607EC0C63020E5D20721F48091FA010B
:1010D000846076C0C83080E5D80719F48091FA01A1
:1010E00027C0CA3090E5D90721F48091FA018061C8
:1010F00067C0CC3020E5D20721F48091FA018062EC
:101100005FC0CE3080E5D80721F48091FA01806479
:1011100057C0C03190E5D90721F48091FA01806869
:101120004FC0C23120E5D20729F48091FA018460D2
:10113000886046C0C33080E5D80721F48091FA0169
:101140008E7F3EC0C53090E5D90721F48091FA0129
:101150008D7F36C0C73020E5D20721F48091FA0197
:101160008B7F2EC0C93080E5D80719F48091FA0131
:1011700026C0CB3090E5D90721F48091FA018F7E0B
:101180001FC0CD3020E5D20721F48091FA018F7D78
:1011900017C0CF3080E5D80721F48091FA018F7B0A
:1011A0000FC0C13190E5D90721F48091FA018F7702
:1011B00007C0C331D04531F48091FA018B7F877F1E
:1011C0008093FA018091FA010E94C21EABC08D2F5C
:1011D00099278F70992781309105D9F49E0123704A
:1011E000332702C0880F991F2A95E2F79C688E0169
:1011F00044E0000F111F4A95E1F700271370802B80
:10120000912B53E0CC0FDD1F5A95E1F7C076DD2717
:101210002FC08230910531F4DC2FCC278E01016F75
:10122000106A80C08330910569F4CE0183709927DC
:1012300001E010E002C0000F111F8A95E2F7C8011B
:101240009C680FC084309105B9F4CE018370992752
:1012500001E010E002C0000F111F8A95E2F7C801FB
:101260009A6823E0CC0FDD1F2A95E1F7C07ED77086
:101270008C010C2B1D2B56C08530910531F4DC2FD1
:10128000CC278E01046F106A4DC0069709F04AC042
:10129000CF71DD27DC2FCC278E01106243C000E028
:1012A00010E040C08E013EC001E810E43BC003E8FE
:1012B00010E438C002EE14E435C009EE14E432C084
:1012C0000AEE14E42FC005EB14E42CC006EB14E482
:1012D00029C007EB14E426C00CEC14E423C00DEC89
:1012E00014E420C003E815E41DC00AE815E41AC0A0
:1012F00002E915E417C004E915E414C001E216E49C
:1013000011C003E216E40EC004E216E40BC005E2CD
:1013100016E408C006E216E405C007E216E402C0BF
:101320000AE216E4C801DF91CF911F910F91089551
:1013300096E0799FF001112494E5899FE00DF11D5D
:101340001124E60FF11DEE0FFF1FE25EFE4F8591A7
:101350009491803E9105E0F4803C910558F58133ED
:10136000910509F46FC048F48932910509F463C00E
:101370008A32910509F46DC072C089339105E9F094
:1013800082389105D1F08533910509F44DC067C0CD
:10139000833E910581F138F4803E9105B9F0823E9B
:1013A0009105D9F05CC0863E910561F1873E9105BB
:1013B000A1F155C00E94560708952091FA0120FD21
:1013C00002C021FF4CC080EE90E049C08091FA013C
:1013D00080FFF9CF89E390E042C08091FA0182FF5B
:1013E0000EC08091FA0184FF03C080E090E037C016
:1013F00083EE90E034C08091FA0182FFF2CF82EE5A
:1014000090E02DC08091FA0183FF0BC08091FA011A
:1014100084FDEBCF87EE90E022C08091FA0183FF3C
:10142000F5CF86EE90E01BC08091FA0185FF07C0E2
:1014300089E290E014C08091FA0185FFF9CF85E33D
:1014400090E00DC08091FA0186FF07C08AE290E02B
:1014500006C08091FA0186FFF9CF81E390E00E94F7
:101460006607089508950C94320A80916E010895DC
:10147000CF93DF9300D01F92CDB7DEB79C01809150
:10148000F101843019F593E099833B832A8390938B
:10149000E9008FEF9091E800815095FD06C095ED31
:1014A0009A95F1F700008111F5CF8091E80085FF52
:1014B0000DC040E050E063E070E0CE0101960E9474
:1014C000A50C8091E8008E778093E8000F900F9034
:1014D0000F90DF91CF910895CF93DF9300D01F92AB
:1014E000CDB7DEB72091F101243021F522E0298328
:1014F0009B838A8383E08093E9008FEF9091E800DB
:10150000815095FD06C095ED9A95F1F70000811187
:10151000F5CF8091E80085FF0DC040E050E063E02A
:1015200070E0CE0101960E94A50C8091E8008E77B4
:101530008093E8000F900F900F90DF91CF91089566
:101540002091F1012430F1F422E02093E9002FEF03
:101550003091E800215035FD06C035ED3A95F1F7A0
:1015600000002111F5CF2091E80025FF0BC040E0DD
:1015700050E065E070E00E94A50C8091E8008E7755
:101580008093E8000895CF93DF93EC019091F101EF
:10159000943009F046C080910C018823D9F08091E5
:1015A0000D018823B9F09093E9008FEF9091E80046
:1015B000815095FD06C095E19A95F1F700008111E3
:1015C000F5CF8091E80085FF2CC040E050E060E15D
:1015D00070E017C081E08093E9008FEF9091E80000
:1015E000815095FD06C095ED9A95F1F700008111A7
:1015F000F5CF8091E80085FF14C040E050E068E03E
:1016000070E0CE010E94A50C8091E8008E77809357
:10161000E80080E1FE01AEE5B1E001900D928A950F
:10162000E1F7DF91CF9108958091F001811109C018
:101630000E943A0E0E94970E8091E200846080938F
:10164000E20008951092F001089508950C9430235B
:101650000E94921C0E9436230E943D110C94330A72
:1016600042E061EC81E00E94B40D42E061EC82E076
:101670000E94B40D42E061EC83E00E94B40D42E1AF
:1016800061EC84E00C94B40D8091F301833009F493
:1016900055C030F4813071F0823009F48EC0089565
:1016A0008A3009F47AC08B3009F460C0893009F0BF
:1016B0009CC020C08091F201813A09F096C08091CF
:1016C000E800877F8093E8008091F6019091F70110
:1016D000892B21F460E18EE591E003C060E080E0B9
:1016E00090E070E00E94F00C8091E8008B7780938E
:1016F000E80008958091F201813209F076C080916E
:10170000F6019091F701009719F0039709F06DC069
:101710008091E800877F8093E8008091E80082FD57
:1017200005C08091F1018111F8CF5FC08091F10077
:1017300080936E018091E8008B7753C08091F20115
:10174000813A09F052C08091F6019091F701892BFE
:1017500009F04BC08091E800877F8093E80080917A
:10176000E80080FFFCCF80910C0136C08091F2012F
:101770008132D9F58091F6019091F701892BA9F575
:101780008091E800877F8093E8000E94E90D8091B6
:10179000F40180930C010C94D6158091F2018132F2
:1017A00021F58091E800877F8093E8000E94E90D91
:1017B0008091F50180936F0108958091F201813A43
:1017C000A1F48091E800877F8093E8008091E80091
:1017D00080FFFCCF80916F018093F1008091E80041
:1017E0008E778093E8000C94E90D089584B7877F85
:1017F00084BF0FB6F894A8958091600088618093AB
:101800006000109260000FBE90E080E80FB6F89480
:1018100080936100909361000FBE0E948C110E9422
:101820003A0E0E94970E8091E20084608093E2005D
:1018300078940E941D110E948E1182E091E00E9416
:1018400038110E941E238091F101853069F40E94B5
:10185000561C8091EF018823B1F30E94841C8823D9
:1018600091F30E948F0CEFCF0E949411ECCF292F9F
:10187000332723303105C9F064F42130310581F07C
:101880002230310509F043C08DE690E02AEE35E0C4
:1018900042C021323105F1F02232310541F137C029
:1018A00082E190E027E536E036C099278130910546
:1018B00041F08230910541F0892B49F5E6EEF5E0E3
:1018C00005C0EEECF5E002C0E6EBF5E0849190E0B7
:1018D0009F0121C06430D8F4E62FF0E0EE0FFF1F27
:1018E000EE5DFE4F2081318189E090E014C06430CC
:1018F00070F470E0FB01EE0FFF1FE65EFE4F2081EB
:101900003181FB01EA5EFE4F808190E004C080E0FF
:1019100090E020E030E0FA0131832083089580E1F7
:1019200089BD82E189BD09B400FEFDCF8091D80058
:101930008F7D8093D8008091E00082608093E000EA
:101940008091E00081FDFCCF0895CF92DF92EF926D
:10195000FF920F931F93CF93DF93EC018B016A01EA
:101960000E94080E811133C0C114D10439F0F60170
:1019700080819181081B190BC80FD91FE12CF12C14
:101980000115110519F18091E80085FD16C08091BF
:10199000E8008E778093E800C114D10449F0F60185
:1019A00080819181E80EF91EF182E08285E00FC00E
:1019B0000E94080E882321F30AC089918093F100C8
:1019C00001501109FFEFEF1AFF0ADACF80E0DF9133
:1019D000CF911F910F91FF90EF90DF90CF900895DE
:1019E0002091F8013091F9012617370748F0611569
:1019F000710539F42091E8002E772093E80001C0AA
:101A0000B90140E061157105A9F12091F10122238E
:101A100009F443C0253009F442C02091E80023FDB9
:101A200040C02091E80022FD32C02091E80020FF54
:101A3000E9CF4091F3002091F20030E0342BFC011B
:101A4000CF016115710559F02830310540F48191BD
:101A50008093F100615071092F5F3F4FF1CF41E05A
:101A60002830310509F040E02091E8002E772093DE
:101A7000E800C8CF4111C9CF0AC08091F101882385
:101A800061F0853061F08091E80083FD0AC08091AB
:101A9000E80082FFF2CF80E0089582E0089583E0BD
:101AA000089581E008952091F8013091F9012617F9
:101AB000370748F06115710539F42091E8002E7759
:101AC0002093E80001C0B901FC0120E06115710517
:101AD00091F18091F101882309F440C0853009F427
:101AE0003FC08091E80083FD3DC08091E80082FD09
:101AF0002FC08091E80080FFE9CF2091F300809112
:101B0000F20090E0922B6115710559F08830910533
:101B100040F424912093F1003196615071090196AF
:101B2000F2CF21E0089709F020E08091E8008E775D
:101B30008093E800CBCF2111CCCF0AC08091F10176
:101B4000882361F0853061F08091E80083FD0AC050
:101B50008091E80082FFF2CF80E0089582E008954E
:101B600083E0089581E00895982F973058F5909379
:101B7000E900981739F07091EC002091ED00509138
:101B8000F00003C0242F762F50E021FF19C03091C0
:101B9000EB003E7F3093EB003091ED003D7F3093C2
:101BA000ED003091EB0031603093EB007093EC006E
:101BB0002093ED005093F0002091EE0027FF07C026
:101BC0009F5FD3CF8F708093E90081E0089580E01C
:101BD00008958091F20187FF11C08091E80082FD95
:101BE00005C08091F1018111F8CF11C08091E8000A
:101BF0008B770BC08091F101882349F08091E80038
:101C000080FFF8CF8091E8008E778093E8000895F8
:101C10002091E4003091E50095E64091EC00842F9E
:101C2000817040FF22C08091E80080FD1CC080913F
:101C3000F101882391F0853091F08091EB0085FDD2
:101C400010C04091E4005091E5004217530729F37A
:101C50009A01915011F784E0089582E0089583E09D
:101C6000089581E0089580E008954091E80042FFE2
:101C7000DECF08950E94A80E0E94B00EE0EEF0E0C4
:101C8000808181608083E8EDF0E080818F778083C0
:101C900019BCA7EDB0E08C918E7F8C9380818F7EF4
:101CA00080831092F00108950F931F93CF93DF93D9
:101CB0000E94A80E0E94B00EC8EDD0E088818F77F8
:101CC000888388818068888388818F7D888319BC18
:101CD0001092F1011092ED011092EF011092EE01BD
:101CE00000EE10E0F80180818B7F80838881816025
:101CF000888342E060E080E00E94B40DE1EEF0E015
:101D000080818E7F8083E2EEF0E08081816080833D
:101D1000808188608083F80180818E7F80838881C4
:101D200080618883DF91CF911F910F910895E8ED35
:101D3000F0E080818F7E8083E7EDF0E0808181603C
:101D4000808384E082BF81E08093F0010C94540E84
:101D5000E8EDF0E080818E7F80831092E2000895AC
:101D60001092DA001092E10008951F920F920FB6C0
:101D70000F9211242F933F934F935F936F937F9311
:101D80008F939F93AF93BF93EF93FF938091E10065
:101D900082FF0BC08091E20082FF07C08091E100CA
:101DA0008B7F8093E1000E941C118091DA0080FFFC
:101DB0001FC08091D80080FF1BC08091DA008E7F09
:101DC0008093DA008091D90080FF0DC080E189BD49
:101DD00082E189BD09B400FEFDCF81E08093F1016D
:101DE0000E94140B05C019BC1092F1010E94220B35
:101DF0008091E10080FF19C08091E20080FF15C052
:101E00008091E2008E7F8093E2008091E200806109
:101E10008093E2008091D80080628093D80019BC42
:101E200085E08093F1010E94260B8091E10084FF00
:101E300030C08091E20084FF2CC080E189BD82E146
:101E400089BD09B400FEFDCF8091D8008F7D8093BD
:101E5000D8008091E1008F7E8093E1008091E200C4
:101E60008F7E8093E2008091E20081608093E200A7
:101E70008091ED01882311F084E007C08091E30098
:101E800087FD02C081E001C083E08093F1010E94E0
:101E9000280B8091E10083FF29C08091E20083FF3D
:101EA00025C08091E100877F8093E10082E08093EC
:101EB000F1011092ED018091E1008E7F8093E100AD
:101EC0008091E2008E7F8093E2008091E200806149
:101ED0008093E20042E060E080E00E94B40D8091D7
:101EE000F00088608093F0000E94250BFF91EF9135
:101EF000BF91AF919F918F917F916F915F914F9122
:101F00003F912F910F900FBE0F901F9018951F9229
:101F10000F920FB60F9211242F933F934F935F931D
:101F20006F937F938F939F93AF93BF93CF93DF93E1
:101F3000EF93FF93C091E900CF708091EC00D82F10
:101F4000D17080FDD0E81092E9008091F000877F89
:101F50008093F00078940E94CB0F1092E90080915A
:101F6000F00088608093F000CD2BCF70C093E90023
:101F7000FF91EF91DF91CF91BF91AF919F918F91A1
:101F80007F916F915F914F913F912F910F900FBE75
:101F90000F901F9018951F93CF93DF93CDB7DEB7A7
:101FA000AA970FB6F894DEBF0FBECDBFE2EFF1E007
:101FB00088E08E0F9091F10091938E13FBCF0E94D9
:101FC000440B8091E80083FF1FC18091F201909142
:101FD000F301492F50E04A30510508F015C1FA01CC
:101FE000EA5AFF4F0C94C724803881F0823809F0F8
:101FF0000BC18091F6018F708093E9008091EB0016
:1020000085FB882780F91092E90006C08091EE01D7
:102010009091EF01911182609091E800977F9093E9
:10202000E8008093F1001092F100C8C0282F2D7FA6
:1020300009F0EAC0882319F0823061F0E5C0809190
:10204000F401813009F0E0C0933009F080E0809322
:10205000EF012BC08091F401811127C08091F6011E
:102060008F7009F4D1C08093E9002091EB0020FF2C
:102070001CC0933021F48091EB00806214C09091D9
:10208000EB0090619093EB0021E030E0A90102C0E9
:10209000440F551F8A95E2F74093EA001092EA0038
:1020A0008091EB0088608093EB001092E9008091B2
:1020B000E800877F86C08111A7C01091F4011F77C7
:1020C0008091E3008078812B8093E3008091E80089
:1020D000877F8093E8000E94E90D8091E80080FFEF
:1020E000FCCF8091E30080688093E300111102C06F
:1020F00082E001C083E08093F10186C08058823085
:1021000008F082C08091F4019091F5018C3D53E07C
:10211000950779F583E08A838AE289834FB7F8943B
:10212000DE01139620E03EE051E2E32FF0E0509311
:102130005700E49120FF03C0E295EF703F5FEF701E
:102140008E2F90E0EA3010F0C79601C0C0968D93B4
:102150009D932F5F243149F74FBF8091E800877F1F
:102160008093E8006AE270E0CE0101960E94F00CD4
:1021700014C0AE014F5F5F4F6091F6010E94370CB3
:10218000BC01892B09F440C09091E800977F90939F
:10219000E80089819A810E94530D8091E8008B7735
:1021A0008093E80031C0803879F58091E800877F1E
:1021B0008093E8008091ED018093F1008091E80028
:1021C0008E778093E8000E94E90D1EC081111CC02B
:1021D0009091F4019230C0F48091E800877F809361
:1021E000E8009093ED010E94E90D8091ED018111CD
:1021F00006C08091E30087FD02C081E001C084E059
:102200008093F1010E94300B8091E80083FF0AC0A7
:102210008091E800877F8093E8008091EB008062E6
:102220008093EB00AA960FB6F894DEBF0FBECDBF29
:10223000DF91CF911F9108950895CF938091F1017F
:102240008823A1F0C091E900CF709091EC00892F14
:10225000817090FD80E8C82B1092E9008091E80021
:1022600083FD0E94CB0FCF70C093E900CF910895FA
:1022700090937501809374010895E0917401F09139
:102280007501309721F00190F081E02D099480E0F4
:102290000895E0917401F0917501309721F002806A
:1022A000F381E02D09940895E0917401F091750196
:1022B000309721F00480F581E02D09940895209154
:1022C0007201309173018217930771F0909373013B
:1022D00080937201E0917401F0917501309721F0C3
:1022E0000680F781E02D09940895209170013091C6
:1022F00071018217930771F09093710180937001BF
:10230000E0917401F0917501309721F00084F1851E
:10231000E02D0994089508950C948B110E94981C47
:102320000E9471050C945A1D9F92AF92BF92CF925A
:10233000DF92EF92FF920F931F93CF93DF9300D022
:1023400000D000D0CDB7DEB70E9489050DE010E0C7
:10235000AA24A394B12C902E802F0E947706980176
:1023600029583E4F6901F901F080F826A1F4015087
:10237000110988F78FEF89838A831B820E94A11C31
:102380008160782F9D838C8349815A816B818D81F7
:102390000E942B122FC09091DA0191FF04C08E830E
:1023A0000E947D068E8125E030E0A501022E01C04D
:1023B000440F0A94EAF7E42E4F21C1F029839A8250
:1023C0008E2191E009F490E09B830E94A11C816022
:1023D000782F9D838C8349815A816B818D810E94E6
:1023E0002B12F6018081E826E08204C021503109D9
:1023F000E0F6BDCF0E944120109176010E943D1170
:102400001817B9F00E943D118093760126960FB6F9
:10241000F894DEBF0FBECDBFDF91CF911F910F911A
:10242000FF90EF90DF90CF90BF90AF909F900C9473
:10243000330A26960FB6F894DEBF0FBECDBFDF91EC
:10244000CF911F910F91FF90EF90DF90CF90BF90B1
:10245000AF909F900895CF93DF93CDB7DEB72B97C2
:102460000FB6F894DEBF0FBECDBF4F835887698784
:102470007A878B87DE01119686E0FD0111928A959D
:10248000E9F785E0FE01379601900D928A95E1F714
:1024900049815A816B817C818D819E810E94741853
:1024A0002B960FB6F894DEBF0FBECDBFDF91CF9154
:1024B0000895CF93882309F4C2C0C82F823859F4F5
:1024C0000E943D1181FDBBC089E30E944E1B0E940A
:1024D0001B1C89E30CC0833879F40E943D1180FDF8
:1024E000AEC083E50E944E1B0E941B1C83E50E9428
:1024F000901BCF910C941B1C843859F40E943D1101
:1025000082FD9DC087E40E944E1B0E941B1C87E435
:10251000EECF8CEF8C0F813A48F48C2F0E948322EF
:1025200081118DC08C2F0E944E1BE3CF80E28C0F57
:10253000883048F4C77081E001C0880FCA95EAF777
:102540000E94D41BD6CF8BE58C0F833078F4C53A2C
:1025500029F0C63A31F083E890E005C081E890E0C8
:1025600002C082E890E0CF910C945F1188E58C0F57
:10257000833108F064C0C83A39F1C93A41F1CA3A26
:1025800049F1CB3A51F1CC3A59F1CD3A61F1C03B26
:1025900069F1CE3A71F1CF3A79F1C13B81F1C23B99
:1025A00089F1C33B91F1C43B99F1C53BA1F1C63B15
:1025B000A9F1C73BB1F1C83BB9F1C93BC1F1CA3B75
:1025C000C9F180E090E038C082EE90E035C089EE3D
:1025D00090E032C08AEE90E02FC085EB90E02CC0F6
:1025E00086EB90E029C087EB90E026C08CEC90E071
:1025F00023C08DEC90E020C083E891E01DC08AE804
:1026000091E01AC082E991E017C084E991E014C01A
:1026100081E292E011C083E292E00EC084E292E097
:102620000BC085E292E008C086E292E005C087E236
:1026300092E002C08AE292E0CF910C947511CF91A2
:102640000895882309F44BC0823859F40E943D1143
:1026500081FF45C089E30E944E1B0E941B1C89E339
:102660000CC0833871F40E943D1180FF38C083E5AF
:102670000E944E1B0E941B1C83E50E94901B0C9421
:102680001B1C843859F40E943D1182FF28C087E446
:102690000E944E1B0E941B1C87E4EFCF9CEF980FFB
:1026A000913A58F390E2980F983050F4877091E087
:1026B00001C0990F8A95EAF7892F0E94DA1BDFCFB4
:1026C0009BE5980F933020F480E090E00C945F112C
:1026D000885A833120F480E090E00C9475110895BD
:1026E000882321F00E94D41B0C941B1C089588237E
:1026F00021F00E94DA1B0C941B1C08957F928F928C
:102700009F92AF92BF92CF92DF92EF92FF920F9380
:102710001F93CF93DF931F92CDB7DEB77C01C62EF8
:10272000772EFC01058102950F70128111110E9414
:10273000F11B0E94471B882379F0112369F080E286
:102740008C0D883048F082E00E94301B0E94471BAD
:1027500091E0D82ED92601C0D12CE72DE295EF705B
:10276000F0E0E05AFF4F0C94C724872D807F072D9F
:102770000F70882311F00295007F112389F0002348
:1027800009F490C180E28C0D883020F4802F0E94E3
:10279000D41B03C0802F0E94E41B0E941B1C82C11B
:1027A0008C2D0E942113002309F495C180E28C0D29
:1027B000883020F4802F0E94DA1B03C0802F0E94F3
:1027C000EA1B0E941B1C87C1972D907F872D8F705D
:1027D000903211F08295807FCC2021F0F1E0CF166D
:1027E000B1F01EC0112349F0002309F414C10130D7
:1027F00009F011C10E94041C6EC1002319F00130C0
:1028000009F469C189830E94071C89810AC11123C7
:1028100021F0023008F05FC1FEC001115CC101C1AE
:10282000112321F0002309F4F6C03CC1002309F470
:10283000F8C03EC1872D86958695837090E00097FD
:1028400019F0019761F047C1112321F08C2D972DCC
:10285000937002C080E090E00E945F113CC11123A0
:1028600021F08C2D972D937002C080E090E00E94A3
:10287000751131C18C2D112319F00E94491F02C01E
:102880000E94B11F0E94362026C1872D837009F057
:1028900052C0111120C18C2D829586958770880FAA
:1028A000880F9C2D9F70892E912CA12CB12C082E65
:1028B00004C0880C991CAA1CBB1C0A94D2F7C4FE45
:1028C00014C00FE010E020E030E0B901A80104C01E
:1028D000440F551F661F771F8A95D2F7CB01BA01A7
:1028E000609570958095909503C060E070E0CB0195
:1028F000272D26952695237030E02230310569F08A
:102900002330310589F0682979298A299B292130CA
:10291000310571F00E94BC19DEC0682979298A2925
:102920009B290E94D819D7C00E94BC19C501B401C7
:102930000E94A019D0C0112319F0872D817001C009
:102940008695882309F4C7C08C2D8295869587705B
:10295000880F880F9C2D9F70892E912CA12CB12C53
:10296000082E04C0880C991CAA1CBB1C0A94D2F720
:10297000C4FE14C00FE010E020E030E0B901A8016F
:1029800004C0440F551F661F771F8A95D2F7CB01ED
:10299000BA01609570958095909503C060E070E0F5
:1029A000CB01272D269526952370422F50E04230EB
:1029B000510569F04330510589F0682979298A2940
:1029C0009B294130510571F00E94961A84C06829F4
:1029D00079298A299B290E94B21A7DC00E94961AE1
:1029E000C501B4010E947A1A76C08C2D90E0FC01DA
:1029F000E05EF109E531F10508F050C0E059FF4F04
:102A00000C94C7240C2D0F70872D8F71112331F07A
:102A10000E94131A802F0E9470135DC00E94341A06
:102A2000802F0E94771357C0112339F0011153C032
:102A3000872D8F710E94591A4EC0023008F04BC08A
:102A4000F7CF112339F0872D8F710E94131A43C0DD
:102A50001123C9F3872D8F710E94341A3CC01123B2
:102A600029F0872D8F710E94FE1935C00E94F4193C
:102A700032C0112351F0172D1F71812F0E94131A9C
:102A800063E0812F0E94271B26C081E00E94301B3B
:102A9000023008F182E00E94301B1DC0112331F08A
:102AA000002389F28C2D0E94591215C0002391F247
:102AB0008C2D0E9421130FC0472D4F706C2DC70124
:102AC0000E941B040E94181906C0472D4F706C2DE0
:102AD000C7010E944307DD20F9F00E94231B80FDFF
:102AE0001BC0F70112820E941D1B0E94131AC7010E
:102AF0000E949B150E941D1B0F90DF91CF911F918B
:102B00000F91FF90EF90DF90CF90BF90AF909F908C
:102B10008F907F900C94341A0F90DF91CF911F917A
:102B20000F91FF90EF90DF90CF90BF90AF909F906C
:102B30008F907F9008950F931F93CF93DF93EC01B5
:102B4000888199812B813C81232BB9F09F3F11F41F
:102B50008F3F99F0CE010E949B06882371F0688117
:102B600079818A810E94191B8C010E94CE1A0E94D1
:102B70009519B801CE010E947E13DF91CF911F916C
:102B80000F9108950E94F11B0E94011C0E94C61B18
:102B90000E941B1C0E94E6200E94362080E090E0EC
:102BA0000E945F1180E090E00C9475110E94E11B7F
:102BB0000C94C2150E940E1B292F22952F7030E015
:102BC0002C3031054CF42A3031056CF42250310997
:102BD00022303105A8F407C02C30310569F02F30C0
:102BE000310551F00DC0803F69F018F4803E40F48B
:102BF00009C0843F29F406C093FB882780F9089513
:102C000080E0089581E00895CF93DF9300D000D055
:102C10001F92CDB7DEB70F900F900F900F900F90CF
:102C2000DF91CF910895CF93DF9300D000D000D0F3
:102C3000CDB7DEB726960FB6F894DEBF0FBECDBF78
:102C4000DF91CF9108951F93CF93DF93C0918501BA
:102C500016E080918601C81799F0D0E01C9FF00122
:102C60001D9FF00D1124E957FE4F40815181628173
:102C70007381848195810E9413162196C770E9CFD4
:102C8000DF91CF911F9108954091B7015091B80104
:102C90006091B9017091BA018091BB019091BC0122
:102CA0000C9413168091BC0182958F7009F054C06A
:102CB0008091B901882309F44FC080918501A091CA
:102CC00086016091B7017091B8014091BA015091AD
:102CD000BB01B6E08A1709F43FC090E041155105E9
:102CE000C1F17F3F11F46F3FA1F1B89FF001B99F8F
:102CF000F00D1124E957FE4F218172132AC0208163
:102D0000621327C02281211124C02381348124171A
:102D1000350710F421503109241B350B283C3105AF
:102D2000C0F42091BC012F7020612093BC0126E0EB
:102D3000289FF001299FF00D1124E457FE4F808158
:102D40008F708061808387EB91E00E949B150C94CB
:102D5000231601968770BECF0895CF92DF92EF922F
:102D6000FF920F931F93CF93DF93CDB7DEB7629798
:102D70000FB6F894DEBF0FBECDBF8C0185E0F80121
:102D8000DE011D9601900D928A95E1F7D8014C91D4
:102D900011965C91119712966C9112971396CD90A3
:102DA000DC9014973091B7017091B8018091BA010D
:102DB0009091BB01009709F46BC17F3F19F43F3F2D
:102DC00009F466C1E090B901EE2009F4C0C0209179
:102DD000BC01C816D90628F0F601E81BF90BCF0193
:102DE00004C0809590958C0D9D1DFF24F394883C24
:102DF000910578F0F12C207F09F0C6C07C2DD98A8E
:102E0000C88A89890E94041687EB91E00E949B156D
:102E1000B1C0822F807F09F046C0751314C03413EF
:102E200012C0611110C02F7020612093BC010E945C
:102E3000441687EB91E00E949B158091BC01D8015C
:102E400015968C932EC0CD2819F15F3F11F44F3F9A
:102E5000F9F0F62E61111CC0809185012091860148
:102E600036E0821709F45AC090E0389FF001399F8C
:102E7000F00D1124E957FE4F7181571306C0708180
:102E8000471303C07281711103C001968770E9CFA7
:102E9000F62E662309F418C18091BC0181608093ED
:102EA000BC01F12C11C1751308C0341306C06111A7
:102EB00004C08091BC01D801C3C04D875E878D8559
:102EC0009E856A8B0E94DA156A898823E1F1662360
:102ED000D1F12091BC01822F82958F7090E00297F2
:102EE00074F08091B7019091B80198878F8319860B
:102EF000DB86CA862C87CE0107960E949B1586E04A
:102F0000F801A7EBB1E001900D928A95E1F70E94DC
:102F100052160E944416FF24F394D6C04D875E8754
:102F20008D859E850E940E1B292F22952F7030E0E3
:102F3000223031050CF0BCC09F7009F0B6C0805E35
:102F4000883008F4C1C0C8010E949B15E4CFC816A0
:102F5000D90608F453C0F601E81BF90BCF01883CF1
:102F6000910508F450C0F12C7C2DD98AC88A898932
:102F70000E940416E7EBF1E086E0DF011D928A95DE
:102F8000E9F70E944416A0C0751314C0341312C090
:102F9000611110C08091BC01F8018583C8010E94B5
:102FA0009B1586E0E7EBF1E0DF011D928A95E9F7DA
:102FB000FE2C8AC04D875E878D859E856A8B0E9418
:102FC000DA156A89882309F4BECF662309F4BBCFDA
:102FD0002091BC01822F82958F7090E002970CF4B3
:102FE0008ECF8091B7019091B8019A8389831B821B
:102FF000DD82CC822E83CE0101967FCF8095909585
:103000008C0D9D1DACCFF62E662309F49CCF751355
:103010002EC034132CC02091BC0120FD1FC0822F74
:1030200082958F70D9F0D80115962C9315978F3013
:1030300049F08F5F982F9295907F822F8F70892B08
:1030400015968C93C8010E949B1586E0F801A7EBAA
:10305000B1E001900D928A95E1F793CF86E0F801F7
:10306000A7EBB1E001900D928A95E1F72DC04D8755
:103070005E878D859E850E94DA15811140CF8091F3
:10308000BC0181608093BC01C8010E949B151CC0DB
:10309000662309F458CF4D875E878D859E850E94F3
:1030A000DA15882309F44FCF2ACF811148CF0CC0FD
:1030B000243031050CF047CF9F7009F440CFF80160
:1030C0009581907F09F03BCF8F2D62960FB6F894D3
:1030D000DEBF0FBECDBFDF91CF911F910F91FF904B
:1030E000EF90DF90CF9008951F93CF93DF93CDB7EC
:1030F000DEB72C970FB6F894DEBF0FBECDBF4F835F
:10310000588769877A878B879C87CE0107960E94AC
:10311000AD16882369F08F8198852A853B85232BFE
:10312000F1F19F3F09F063C08F3F09F060C037C0E5
:1031300086E0FE013796DE01119601900D928A9588
:10314000E1F76F817885EA85FB85309741F17F3F14
:1031500011F46F3F21F12091860130E0C901019601
:10316000877099274091850150E08417950709F4ED
:1031700047C069837A83FD83EC8396E0929FD001F8
:10318000939FB00D1124A957BE4FFE0131960190B7
:103190000D929A95E1F7809386010E94231616E01E
:1031A00080918501909186018917C1F1189FC00116
:1031B000112489579E4F0E94AD16882379F1E09122
:1031C00085011E9FF0011124E957FE4F4081518176
:1031D00062817381848195810E941316809185019B
:1031E00090E001968770992780938501D9CF4F8110
:1031F000588569857A858B859C850E941316CFCF6B
:103200000E94D6151092860110928501E7EBF1E03D
:1032100086E0DF011D928A95E9F7C1CF2C960FB6A3
:10322000F894DEBF0FBECDBFDF91CF911F910895FF
:10323000EF92FF920F931F93CF93DF938C01892B13
:1032400009F46CC0F12CEE24E394E8012196F80116
:103250008491843740F4843008F051C0813081F08B
:10326000823019F15BC0853709F444C0A8F19CE7AE
:10327000980F903708F052C08F770E94211341C0F9
:103280000E5F1F4FFE01C49180E28C0F883048F41E
:10329000C7708E2D01C0880FCA95EAF70E94F41BF3
:1032A00014C08C2F0E9459122DC00E5F1F4FFE01BB
:1032B000C49180E28C0F883058F4C7708E2D01C005
:1032C000880FCA95EAF70E94FA1B0E941B1C1AC0BD
:1032D0008C2F0E94211316C00E5F1F4FFE01C49158
:1032E000CC2381F08FE99FE00197F1F700C0000047
:1032F000C150F6CF0E5F1F4FFE01F49003C00E9435
:1033000059128E018F2D882309F49FCFEFE9FFE03A
:103310003197F1F700C000008150F5CFDF91CF91D8
:103320001F910F91FF90EF90089508956093C10150
:103330007093C2018093C3019093C4010C94C21591
:103340000F931F930091C1011091C2012091C301FD
:103350003091C401DC01CB01802B912BA22BB32B2C
:103360008093C1019093C201A093C301B093C401A3
:103370001F910F910C94C2150F931F930091C101DF
:103380001091C2012091C3013091C401DC01CB0135
:1033900080239123A223B3238093C1019093C20180
:1033A000A093C301B093C4011F910F910C94C21557
:1033B0000F931F930091C1011091C2012091C3018D
:1033C0003091C401DC01CB0180279127A227B327CC
:1033D0008093C1019093C201A093C301B093C40133
:1033E0001F910F910C94C2151092BD011092BE0155
:1033F0001092BF011092C0010C94C21541E050E040
:1034000060E070E004C0440F551F661F771F8A9567
:10341000D2F74093BD015093BE016093BF017093FA
:10342000C0010C94C21541E050E060E070E004C0BF
:10343000440F551F661F771F8A95D2F78091BD01F3
:103440009091BE01A091BF01B091C001482B592BB2
:103450006A2B7B2B4093BD015093BE016093BF014B
:103460007093C0010C94C21541E050E060E070E040
:1034700004C0440F551F661F771F8A95D2F74095E9
:103480005095609570958091BD019091BE01A0917D
:10349000BF01B091C001482359236A237B23409385
:1034A000BD015093BE016093BF017093C0010C94A5
:1034B000C21541E050E060E070E004C0440F551FC9
:1034C000661F771F8A95D2F78091BD019091BE014A
:1034D000A091BF01B091C001482759276A277B27D7
:1034E0004093BD015093BE016093BF017093C00132
:1034F0000C94C2150F931F930091BD011091BE0152
:103500002091BF013091C001DC01CB01802B912BB8
:10351000A22BB32B8093BD019093BE01A093BF015A
:10352000B093C0011F910F910C94C2150F931F937C
:103530000091BD011091BE012091BF013091C001E9
:10354000DC01CB0180239123A223B3238093BD010F
:103550009093BE01A093BF01B093C0011F910F9142
:103560000C94C2150F931F930091BD011091BE01E1
:103570002091BF013091C001DC01CB018027912750
:10358000A227B3278093BD019093BE01A093BF01F2
:10359000B093C0011F910F910C94C2150895CF9262
:1035A000DF92EF92FF920F931F93CF93DF938C01E3
:1035B000C090C101D090C201E090C301F090C4015D
:1035C0008091BD019091BE01A091BF01B091C00159
:1035D000C82AD92AEA2AFB2ACFE1D0E0D701C601BE
:1035E0000C2E04C0B695A795979587950A94D2F7A7
:1035F00080FF06C0B8018C2F0E949809019721F422
:10360000219760F780E001C08C2FDF91CF911F914F
:103610000F91FF90EF90DF90CF900895CF93DF93BD
:10362000EC010E94CF1ABE010E949809DF91CF9150
:103630000895CB010E940E1B08958091C5018595C8
:103640008595859508958091C5018770089598E0C6
:10365000899F90011124262B2093C5010C94131AE5
:103660002091C501809582238093C501982F977082
:1036700069F430E0482F082E000C550B241735074D
:1036800029F08595859585950C94341A0895909127
:10369000C501977081E009F480E0089590910C01D4
:1036A000992321F090910D01911109C020910E01F3
:1036B00030910F01F90132969FEF40E01FC0982F23
:1036C0009695969596959F3050F5E0910E01F09164
:1036D0000F01E90FF11D877021E030E0A90102C060
:1036E000440F551F8A95E2F7CA019181892B818386
:1036F00008959F3F39F04F5F4E3041F0519158137C
:10370000F8CF0DC05111F7CF942FF5CF9F3F39F06F
:10371000F901E90FF11D97FDFA9582830895089547
:1037200090910C01992321F090910D01911109C004
:1037300020910E0130910F01F9013296205F3F4F29
:103740001FC0982F9695969596959F30F0F4E0912E
:103750000E01F0910F01E90FF11D877021E030E0BB
:10376000A90102C0440F551F8A95E2F7CA0180954E
:1037700091818923818308953196E217F30729F017
:1037800090819813F9CF1082F7CF089581E090E0EF
:10379000E0910E01F0910F01E80FF91F10820196E0
:1037A00080319105A9F708959091D901892B8093D3
:1037B000D901089580959091D90189238093D901E9
:1037C00008951092D90108959091D801892B809382
:1037D000D801089580959091D80189238093D801CC
:1037E00008951092D80108959091D701892B809364
:1037F000D701089580959091D70189238093D701AF
:1038000008951092D70108958093C60108951092EB
:10381000C601089580910E0190910F01FC0131962F
:103820009C01205F3F4F80E0919191118F5FE217E3
:10383000F307D1F70895E0910E01F0910F01809107
:10384000D9018083E0910E01F0910F019081809168
:10385000D801892B8083E0910E01F0910F019081B6
:103860008091D701892B80838091C601882361F0E4
:10387000E0910E01F0910F019081892B80830E94CD
:103880000A1C81111092C60180910E0190910F01C6
:103890000C94491120E0009739F0AC0141505109D6
:1038A000842395232F5FF7CF822F08958091F10114
:1038B000843039F11092DB0120E488E190E00FB60A
:1038C000F894A895809360000FBE2093600080E07C
:1038D0000E94330A83B7817F846083BF83B781608E
:1038E00083BF7894889583B78E7F83BF0FB6F89493
:1038F000A8958091600088618093600010926000BC
:103900000FBE0895089508950E94821C0E948905A3
:103910000E94831C0E947E0691E0811101C090E00C
:10392000892F08950E94D6150E943D110C94330AE8
:1039300082E084BD93E095BD9AEF97BD80936E00C1
:1039400008952FB7F8948091DC019091DD01A0914A
:10395000DE01B091DF012FBF0895CF92DF92EF9289
:10396000FF920F931F932FB7F8944091DC01509171
:10397000DD016091DE017091DF012FBF6A017B01E3
:10398000EE24FF248C0120E030E0C016D106E206D0
:10399000F30610F4415051099A01281B390BC90153
:1039A0001F910F91FF90EF90DF90CF9008951F929D
:1039B0000F920FB60F9211248F939F93AF93BF93E3
:1039C0008091DC019091DD01A091DE01B091DF01D9
:1039D0000196A11DB11D8093DC019093DD01A093A0
:1039E000DE01B093DF01BF91AF919F918F910F9056
:1039F0000FBE0F901F9018950E943A0EF8942FEF6B
:103A000087EA91E6215080409040E1F700C0000035
:103A100087E090EBDC018093FB019093FC01A09385
:103A2000FD01B093FE019CE088E10FB6F894A895E3
:103A3000809360000FBE90936000FFCFEF92FF92E3
:103A40000F931F93CF93DF93D82FCDE08C2F0E943D
:103A5000770605E010E0E82EF12CC701002E02C029
:103A6000959587950A94E2F780FF09C0602F7C2F17
:103A700080E00E944407D81302C081E006C00150D4
:103A8000110958F7C15010F780E0DF91CF911F91D5
:103A90000F91FF90EF900895CF93C82F8CE20E9472
:103AA0001E1D882321F08C2FCF910C941E1D80E0C9
:103AB000CF910895CF930E94A11E811102C00E9450
:103AC000871EC5E6C15049F00E9489058FE39CE935
:103AD0000197F1F700C00000F5CF89E20E944C1D6C
:103AE000811113C18AE20E944C1D81110E94871E20
:103AF00085E00E944C1D81110E94FC1C0E94AC1E9E
:103B00008093DA0187E00E944C1D8823A9F18BE1A4
:103B10000E944C1D882351F08091DA0181FB2227FD
:103B200020F991E0922790FB81F90EC08EE00E946F
:103B30004C1D882361F08091DA0182FB222720F955
:103B400091E0922790FB82F98093DA0115C080E121
:103B50000E944C1D9091DA01882341F093FB2227AB
:103B600020F981E0822780FB93F904C0892F80959A
:103B700080FB90F99093DA018091DA010E94B01EE7
:103B80000E94BE1E8093FA0180EE0E944C1D882385
:103B900041F08091FA01982F909590FB80F98093E5
:103BA000FA0189E30E944C1D882359F08091FA01A3
:103BB00081FB222720F991E0922790FB81F98093E5
:103BC000FA0182EE0E944C1D882359F08091FA017F
:103BD00082FB222720F991E0922790FB82F98093C3
:103BE000FA0186EE0E944C1D882359F08091FA015B
:103BF00083FB222720F991E0922790FB83F98093A1
:103C0000FA0183EE0E944C1D882359F08091FA013D
:103C100084FB222720F991E0922790FB84F980937E
:103C2000FA0185E30E944C1D882359F08091FA0126
:103C300085FB222720F991E0922790FB85F980935C
:103C4000FA0181E30E944C1D882359F08091FA010A
:103C500086FB222720F991E0922790FB86F980933A
:103C6000FA0181E10E944C1D882359F08091FA01EC
:103C700087FB222720F991E0922790FB87F9809318
:103C8000FA018091FA010E94C21E8091FA0187FB1D
:103C9000882780F980930D0187E20E944C1DC82F70
:103CA0008EE10E944C1D8111C2608FE10E944C1D6B
:103CB0008111C46080E20E944C1D8111C86081E2C4
:103CC0000E944C1D8111C06182E20E944C1D811135
:103CD000C06283E20E944C1D8111C06484E20E9494
:103CE0004C1D882311F0C06802C0CC2329F08C2F12
:103CF0000E94B91E6C2F03C00E94B51E682F70E091
:103D000080E090E0CF910C949619CF9108956DEEDC
:103D10007EEF80E090E00E94012560E082E090E08C
:103D20000E94EF2460E083E090E00E94EF2460E0D6
:103D300084E090E00E94EF2460E085E090E00C9445
:103D4000EF2480E090E00E94E92421E08D3E9E4F28
:103D500009F020E0822F089582E090E00C94E124A5
:103D6000682F82E090E00C94EF2483E090E00C94C4
:103D7000E124682F83E090E00C94EF2484E090E04D
:103D80000C94E124682F84E090E00C94EF2480915F
:103D9000E20180FF0BC06091130185E0689FB001D4
:103DA000112475956795759567952BC081FF09C09E
:103DB0006091130185E0689FB001112475956795A6
:103DC00020C082FF07C06091130185E0689FB001A9
:103DD000112417C09091E3019923D1F06091120151
:103DE000961788F72091130185E0289F90011124F0
:103DF000929FA001939F500D112470E0CA010E9470
:103E0000B3246038710540F46115710539F002C0C2
:103E100065E070E0862F08958FE7089581E00895AA
:103E20008091E20180FF08C06091110170E07595FA
:103E300067957595679521C081FF06C06091110156
:103E400070E07595679519C082FF04C060911101FB
:103E500070E010C09091E3019923C1F060911001CE
:103E60009617A0F780911101899FC001112470E07D
:103E70000E94B3246038710528F46115710521F0A2
:103E8000862F08958FE7089581E0089561E070E03E
:103E9000F4CF803F21F40E94C71E819504C0813F6A
:103EA00029F40E94C71E8093E6010895823F21F401
:103EB0000E94C71E819504C0833F29F40E94C71E3B
:103EC0008093E5010895893F19F40E94101F05C0F1
:103ED0008A3F31F40E94101F81958093E701089575
:103EE0008B3F21F40E94101F819504C08C3F29F460
:103EF0000E94101F8093E8010895843F21F480916F
:103F0000E401816017C0853F21F48091E401826063
:103F100011C0863F21F48091E40184600BC0873F8B
:103F200021F48091E401886005C0883F31F48091DC
:103F3000E40180618093E40108958D3F21F4809134
:103F4000E20181600BC08E3F21F48091E20182602A
:103F500005C08F3F29F48091E20184608093E201E3
:103F60000895803F39F48091E60187FF6CC010927C
:103F7000E60169C0813F29F48091E6011816BCF37F
:103F800062C09091E501823F29F497FF5CC01092D6
:103F9000E50159C0833F19F41916CCF354C0893F89
:103FA00041F48091E70118160CF04DC01092E70122
:103FB0004AC08A3F29F48091E70187FF44C0F6CFC9
:103FC0008B3F39F48091E80187FF3DC01092E801F2
:103FD0003AC08C3F29F48091E8011816BCF333C035
:103FE000843F21F48091E4018E7F17C0853F21F446
:103FF0008091E4018D7F11C0863F21F48091E4011E
:104000008B7F0BC0873F21F48091E401877F05C03F
:10401000883F31F48091E4018F7E8093E40113C0E6
:104020008D3F21F48091E2018E7F0BC08E3F21F401
:104030008091E2018D7F05C08F3F29F48091E201DC
:104040008B7F8093E2018091E50181110EC0809108
:10405000E60181110AC08091E701811106C08091BB
:10406000E801811102C01092E301089584EE91E00D
:104070000E9454110E94A11C9093E1018093E001E1
:1040800008951F93CF93DF938091E0019091E10118
:104090000E94AD1CAC019091E301992321F0209185
:1040A000140130E006C0209115018AE0289F90019C
:1040B00011244217530708F485C08091E501C0918F
:1040C000E601D091E7011091E801811107C0C1110B
:1040D00075C0D11173C0111171C074C09F3F19F028
:1040E0009F5F9093E301181624F40E94C71E8093EB
:1040F000E5018091E50187FF05C00E94C71E8195FB
:104100008093E5011C1624F40E94C71E8093E601EB
:104110008091E60187FF05C00E94C71E81958093AC
:10412000E6016091E501662331F1C091E601CC23FF
:1041300011F1062E000C770B880B990B0E94BA2305
:1041400023E333E343E35FE30E941E240E948223C0
:104150006093E5016C2FCC0F770B880B990B0E94B5
:10416000BA2323E333E343E35FE30E941E240E9468
:1041700082236093E6011D1624F40E94101F809391
:10418000E7018091E70187FF05C00E94101F81951C
:104190008093E701111624F40E94101F8093E80118
:1041A0008091E80187FF05C00E94101F81958093D0
:1041B000E801DF91CF911F910C9436209F3F09F0C9
:1041C0008FCF97CFDF91CF911F910895E4EEF1E06B
:1041D00085E0DF011D928A95E9F71092E3011092C4
:1041E000E2010895833081F128F4813059F0823062
:1041F000D1F00895853009F449C0B8F1863009F44A
:1042000056C0089580911501262F30E0280F311DEA
:104210002F3F310524F4680F6093150108958FEF47
:1042200080931501089580911401262F30E0280F06
:10423000311D2F3F310524F4680F60931401089558
:104240008FEF80931401089580911301262F30E0A1
:10425000280F311D2F3F310524F4680F609313019F
:1042600008958FEF80931301089580911201262FF6
:1042700030E0280F311D2F3F310524F4680F609383
:10428000120108958FEF809312010895809111011A
:10429000262F30E0280F311D2F3F310524F4680F01
:1042A0006093110108958FEF80931101089580911B
:1042B0001001262F30E0280F311D2F3F310524F447
:1042C000680F6093100108958FEF80931001089597
:1042D000833011F128F4813049F0823091F0089553
:1042E000853081F120F18630C1F10895809115016A
:1042F000681720F4861B809315010895109215010C
:10430000089580911401681720F4861B809314018E
:10431000089510921401089580911301681720F4F4
:10432000861B8093130108951092130108958091C4
:104330001201681720F4861B8093120108951092D1
:104340001201089580911101681720F4861B809353
:1043500011010895109211010895809110016817BC
:1043600020F4861B80931001089510921001089587
:104370000F931F938D3109F46BC008F03FC08E304E
:1043800009F47FC0C0F4873009F469C068F486304E
:1043900009F0B1C08091DA01817F8E7F8093DA01CC
:1043A00081E08093EA01A8C0883009F4A2C08B3074
:1043B00009F49FC0A0C0863109F49BC078F4803115
:1043C00009F472C0813109F096C00E94D61590910F
:1043D0000D0181E0892780930D018BC0893109F49B
:1043E00088C08B3109F087C08091DA0181FB2227D8
:1043F00020F991E0922790FB81F94CC0853309F4B4
:1044000070C048F4873209F46CC008F459C089328E
:1044100009F467C070C0833438F48A3308F04EC0A2
:10442000883309F466C067C0833409F45AC08834FD
:1044300009F061C00E94D6150FEF13ED20E3015083
:1044400010402040E1F700C000000E94FC1C51C059
:104450000E943C230E943D110E94330A4AC0909161
:10446000DA01892F8095817080FB90F929F09660A0
:1044700098609093DA0140C0997F977F9093DA011A
:1044800038C08091DA0182FB222720F991E092273F
:1044900090FB82F98093DA01992359F18091DA0136
:1044A00081608093DA0125C08091DA0183FB2227A5
:1044B00020F991E0922790FB83F9ECCF895301C05A
:1044C0008D5141E050E060E070E08A019B0104C042
:1044D000000F111F221F331F8A95D2F7C901B8019F
:1044E00004C061E070E080E090E00E9496190E94B4
:1044F000D61581E001C080E01F910F91089580E002
:10450000089580E00895CF93C82F8091EA0181300B
:1045100079F018F08230E9F187C0E0910E01F09156
:104520000F018081813169F0823209F07FC009C0BA
:10453000E0910E01F0910F018081813111F0823202
:1045400061F48C2F0E947F22811104C08C2F0E9465
:10455000B8211DC081E090E01AC08C2F0E948122FA
:10456000811114C0C43179F048F4CB3079F0C031F6
:1045700009F060C082E08093EA0108C0C93219F0F6
:10458000C83321F057C01092EA0154C081E0817015
:1045900053C0C93289F118F5C43171F1A8F4C7309C
:1045A00009F046C08AE08093150194E190931401CC
:1045B00093E0909313018093120188E0809311019E
:1045C00088E28093100134C0CE51C63088F5EC2FBC
:1045D000F0E0E65DFE4F80818093E90129C0CE3492
:1045E000E9F020F4CB3421F56AE013C0C13579F04D
:1045F000C235F1F461E00DC08091E901882319F022
:104600001092E90115C081E08093EA0115C061E0D4
:1046100006C08091E9010E94F2200AC06AE0809100
:10462000E9010E94682104C01092EA0180E004C000
:1046300081E002C080E0ABCFCF910895E1E8F0E0E7
:104640008081886080838081816080838FB7F894C7
:1046500093E09093890090ED909388008FBF089528
:10466000EFE6F0E08081826080830895EFE6F0E07D
:1046700080818D7F80830895EFE6F0E0908182E075
:104680008927808308951F920F920FB60F921124ED
:104690002F933F934F935F936F937F938F939F934A
:1046A000AF93BF93EF93FF938091EB019091EC0157
:1046B00001969093EC018093EB01811103C082E09D
:1046C0000E94330AE091EC01E695E695F0E0EC59A2
:1046D000F84FE4918091EB018E1303C080E00E94BB
:1046E000330AFF91EF91BF91AF919F918F917F918D
:1046F0006F915F914F913F912F910F900FBE0F904F
:104700001F9018950E9489236894B1110C94182465
:1047100008950E94FD2388F09F5798F0B92F99279C
:10472000B751B0F0E1F0660F771F881F991F1AF09C
:10473000BA95C9F714C0B13091F00E941724B1E0C6
:1047400008950C941724672F782F8827B85F39F0C5
:10475000B93FCCF3869577956795B395D9F73EF435
:1047600090958095709561957F4F8F4F9F4F0895DD
:10477000E89409C097FB3EF49095809570956195FB
:104780007F4F8F4F9F4F9923A9F0F92F96E9BB27B1
:104790009395F695879577956795B795F111F8CF2D
:1047A000FAF4BB0F11F460FF1BC06F5F7F4F8F4F98
:1047B0009F4F16C0882311F096E911C0772321F08E
:1047C0009EE8872F762F05C0662371F096E8862F26
:1047D00070E060E02AF09A95660F771F881FDAF77D
:1047E000880F9695879597F9089557FD9058440F2F
:1047F000551F59F05F3F71F04795880F97FB991F40
:1048000061F09F3F79F087950895121613061406FC
:10481000551FF2CF4695F1DF08C016161706180689
:10482000991FF1CF86957105610508940895E89464
:10483000BB2766277727CB0197F908950E9431247B
:104840000C94A2240E94942438F00E949B2420F00F
:10485000952311F00C948B240C94912411240C9426
:1048600018240E94F52370F3959FC1F3950F50E033
:10487000551F629FF001729FBB27F00DB11D639F12
:10488000AA27F00DB11DAA1F649F6627B00DA11DB8
:10489000661F829F2227B00DA11D621F739FB00D5E
:1048A000A11D621F839FA00D611D221F749F3327CE
:1048B000A00D611D231F849F600D211D822F762F67
:1048C0006A2F11249F5750409AF0F1F088234AF044
:1048D000EE0FFF1FBB1F661F771F881F91505040B0
:1048E000A9F79E3F510580F00C948B240C9418245A
:1048F0005F3FE4F3983ED4F3869577956795B79537
:10490000F795E7959F5FC1F7FE2B880F911D969550
:10491000879597F9089597F99F6780E870E060E0C0
:1049200008959FEF80EC089500240A941616170648
:1049300018060906089500240A9412161306140690
:1049400005060895092E0394000C11F4882352F0F3
:10495000BB0F40F4BF2B11F460FF04C06F5F7F4FAB
:104960008F4F9F4F089597FB072E16F4009407D0A2
:1049700077FD09D00E94CD2407FC05D03EF4909528
:1049800081959F4F0895709561957F4F0895EE0F23
:10499000FF1F0590F491E02D0994AA1BBB1B51E168
:1049A00007C0AA1FBB1FA617B70710F0A61BB70B9F
:1049B000881F991F5A95A9F780959095BC01CD0144
:1049C0000895F999FECF92BD81BDF89A992780B5D7
:1049D0000895A8E1B0E042E050E00C940925262FAC
:1049E000F999FECF92BD81BDF89A019700B40216E5
:1049F00039F01FBA20BD0FB6F894FA9AF99A0FBE93
:104A000008950196272F0E94F0240C94EF24DC01D6
:104A1000CB01FC01F999FECF06C0F2BDE1BDF89AC9
:104A2000319600B40D9241505040B8F70895F89473
:024A3000FFCFB6
:104A32002002350AC30AA00A6C0A380A0101C7011A
:104A420028080A03140A3F4D36392507D806A2065C
:104A52006906FC0515062E06470601020304050633
:044A62000708090038
:00000001FF
